:020000040800F2
:10000000C80D0020D900000829160008291500088D
:1000100000000000000000000000000000000000E0
:10002000000000000000000000000000B7190008F8
:100030000000000000000000B5190008B919000810
:10004000090100080000000009010008090100087A
:100050000901000809010008090100080901000858
:10006000000000000901000809010008090100085A
:10007000090100080901000809010008000000004A
:10008000090100080000000000000000090100084C
:10009000000000000901000809010008090100082A
:1000A000000000000901000800000000090100082C
:1000B000090100080000000000000000C93000082D
:1000C0000448854600F0AEF8004800472F3200088B
:1000D000C046C046C80D00200C4880F308880C4874
:1000E0000168090E0B4A914205D10B480B4901608A
:1000F0000B480C4901600C4880470C480047FEE75C
:10010000FEE7FEE7FEE7FEE7FEE70000C80D002081
:10011000040000001F000000181002400100000051
:100120000000014000000000371A0008C10000086C
:1001300030B50B46014600202022012409E00D467F
:10014000D5409D4205D31D469540491B2546954007
:1001500040191546521E002DF1DC30BDF0B51FB41C
:100160000646002082B005464024019100901BE025
:10017000019922460F46304600F020F8049A059B6C
:10018000801A994110D310461946224600F039F8DA
:10019000361A8F410197224601200021009F00F06E
:1001A00030F838184D4100902046641E0028DFDCEE
:1001B000019B00982946324607B0F0BD10B5202AB1
:1001C00004DB0846203AD040002110BD0B46D34046
:1001D000D0402024A21A91400843194610BDD2B243
:1001E00001E00270401C491EFBD270470022F6E776
:1001F00010B513460A4604461946FFF7F0FF20469D
:1002000010BD10B5202A04DB0146203A91400020A1
:1002100010BD914020239C1A0346E34019439040AF
:1002200010BD0000064C0125064E05E0E36807CC32
:100230002B430C3C98471034B442F7D3FFF744FFEC
:1002400098320008B832000870B58C180578401C48
:100250006B075B0F01D10378401C2A1106D102788D
:10026000401C03E006780E70401C491C5B1EF9D14F
:100270002B0705D40023521E0DD40B70491CFAE73E
:100280000378401CCB1A921C03E01D780D70491CAA
:100290005B1C521EF9D5A142D8D3002070BD0020AE
:1002A000704700207047000010B501210B4801F095
:1002B0004DFF0B490C4B08600A498A6B002102E094
:1002C000545C5C54491C04468142F9D3A2B20649ED
:1002D000024801F04AFC002010BD000090010020FF
:1002E000A0000020100400205406002072B6FEE793
:1002F00070B5044600F0E6F80546601C02D00448DC
:100300000078241800F0DEF8401BA042FAD370BD3C
:10031000A4000020F8B5002303240125BAE02E46EE
:100320009E40B44632407CD00E79B607B60F012EFF
:1003300001D0022E17D186682746B6465E00B74028
:1003400000967646BE43B646CF68009EB7407646D6
:100350003743876046686746BE430F79FF06FF0F45
:100360009F40374347600E79F643B6070ED0C66804
:100370002746B4465E00B646B7406646BE43B4461E
:100380008F687646B74066463743C7600E79B60732
:10039000B60F022E14D1DE08B60036180096366A63
:1003A0005F07B446FE0E0F27B646B7406646BE430B
:1003B000B4460F697646B74066463743009E3762BB
:1003C00006682746B4465E00B646B7406646BE435A
:1003D0000F79B446BF07BF0F7646B740664637432E
:1003E00007604E68B603B60F53D02D4FBE692E433B
:1003F000BE61BE699F08F607F60F2A4EBF00BE1900
:100400000096B6680F27B4469E07360FB646B7402B
:100410006646BE430927FF06B446B84202D100270C
:1004200010E036E0204FB84201D101270AE01F4F0B
:10043000B84201D1022705E01D4FB84201D1032780
:1004400000E005277646B74066463743009EB76012
:10045000184EB6684F689643FF0200D51643154FF5
:10046000BE60FE684F689643BF0200D51643114F29
:10047000FE607E684F689643BF0300D516430D4F5C
:100480007E603E684F689643FF0300D51643094AD5
:1004900016605B1C0A681646DE4000D03FE7F8BDD8
:1004A000001002400000014000040048000800481D
:1004B000000C004800040140002A01D0816170470F
:1004C000816270470148806870470000A4000020E6
:1004D000024881680278891881607047A400002072
:1004E00010B506480168102211430160032000F096
:1004F00007F800F027F8002010BD0000002002409F
:1005000070B504460D4D7D202978C000FFF710FE20
:1005100001460B480068FFF70BFE00F0EDFF0028D6
:1005200009D1042C07D200222146401E00F030F8E9
:1005300000206C6070BD012070BD0000A400002090
:10054000B000002008B50A48816901221143816189
:10055000816911400091C26901040A43C261C06906
:10056000084000900348016810221143016008BD53
:100570000010024000000140002805DBC106C90E42
:1005800001208840014908607047000000E100E058
:1005900010B502F003FE10BD10B50523DB01C31832
:1005A000016801220B241A65A401002300190372BB
:1005B0004031888A10438882888A022210438882C8
:1005C000184610BD704710B50C0606D54907490FEF
:1005D000282461430818103004E0282461430818D7
:1005E000FF30513099B2002A06D0012202730181F6
:1005F000190C4181002010BD00220273C180F9E76F
:1006000028224A4310B512180523DB01C018526A8C
:10061000806D01F0F7FC10BD28224A43121810B576
:100620000523FF32DB010132C018526E806D01F0EC
:100630004CFD10BD70B5CD094907490F0A46282366
:100640005943091801230024002D02D04B741031A6
:1006500002E0FF3151314C700A700522D201851839
:100660002A7C012A06D02B74006802F0B1F92C74A0
:10067000002070BD022070BD70B50A070379120F0B
:100680009A4201D9012070BDCD094907490F0A4698
:1006900028235943091801230024002D02D04B744C
:1006A000103102E0FF3151314C708C700A7005221C
:1006B000D20185182A7C012A06D02B74006802F02A
:1006C0001BFA2C74002070BD022070BDF8B50368C1
:1006D0000D781C46AC46EE00403357048D691B8AEA
:1006E000002F29DA1B192D4C34191B5B9C05A40D16
:1006F000A54203D32B1B8B6102D00DE000238B613D
:10070000634605689E00AB5B254F3B4001277F0396
:100710007B40244F3B43AB53520609D50A7803680C
:1007200095005A5B204E32401E4E403632435A539B
:10073000002C30D00A8929E01B19184C241D3419CB
:100740001B5B9C05A40DA54203D32B1B8B6102D020
:100750000DE000238B61634605689E00AB5B104F84
:100760003B4001277F037B400E4F3B43AB53520678
:1007700009D40A7805689300EA5A0B4E3240094EB4
:1007800040363243EA52002C05D04A894969006854
:10079000234602F0A4FC2046F8BD0000020400003D
:1007A0008FBF0000808000008F8F0000FEB50C46D8
:1007B00007680197054620780090C300A069164697
:1007C0005106844622464037002020323F8A0029C5
:1007D000019974DA7F18C7495918795A8905890D22
:1007E0008C4514D967467F1AA76111D073040AD5C6
:1007F000009B2F689E00BB5BBC46BF4F3B40BF4F7A
:100800003B436746BB531379012B4BD061E1A06199
:100810006178002902D0012911D018E029685022FE
:10082000525A51185A18B34951180A889205920D14
:100830000A800A880123DB031A430A8007E029683B
:100840005022525A51185A18AA49511808806278F1
:100850002968002A02D0012A13D01CE05020405AF7
:1008600040182178C9000918A248001D08180188FD
:100870008905890D018001880122D203114301807D
:1008800009E05022525A51182278D2005218994940
:10089000091D5118088021782846FFF7B1FE700421
:1008A00075D416E163695B186361E3695B18E36102
:1008B0002669236AB34203D33146581A04E041E063
:1008C000002B107101D0194620626078002802D0F8
:1008D00001282AD033E028685022125A10182278B2
:1008E000D20012188348101802889205920D0280D7
:1008F000002908D03E290CD84A08CB0700D0521C4A
:10090000038892020EE002880123DB031A4302806F
:1009100015E04A09CB0600D1521E03889202012637
:10092000F60332431343038009E028685022125A29
:1009300010182278D20012186E48101801808BB25D
:100940002289C2E07F186B49091D5918795A890517
:10095000890D8C4514D367467F1AA76111D07304A3
:100960000AD4009B2F689E00BB5BBC46624F3B4095
:10097000624F3B436746BB531379012B55D0A8E028
:10098000A0616178002903D0012912D019E042E06A
:1009900029685022525A51185A18564951180A8833
:1009A0009205920D0A800A880123DB031A430A800C
:1009B00007E029685022525A51185A184D495118C7
:1009C000088062782968002A02D0012A13D01CE02E
:1009D0005020405A40182178C90009184548001D88
:1009E000081801888905890D018001880122D20338
:1009F0001143018009E05022525A51182278D20046
:100A000052183C49091D5118088021782846FFF7E3
:100A1000F7FD70045DD4207829688200885A364B2F
:100A20001840364B1843885253E063695B18636182
:100A3000E3695B18E3612669236AB34203D3314655
:100A4000581A206204E0002B01D019462062107170
:100A500062782868002A02D0012A2AD033E0502286
:100A6000125A10182278D20012182248001D1018AD
:100A700002889205920D0280002908D03E290CD8E8
:100A80004A08CB0700D0521C038892020EE002886D
:100A90000123DB031A43028015E04A09CB0600D18B
:100AA000521E038892020126F60332431343038049
:100AB00009E05022125A10182278D20012180D485C
:100AC000001D1018018062898BB26169286802F0EC
:100AD00022FB207829688200885A074B303318405F
:100AE0001023584020235840054B184388520020BB
:100AF000FEBD0000020400008F8F000080C00000D7
:100B0000808000004907490F282251430818FF3010
:100B10000130C06E7047F8B5CD094907490F0F463F
:100B200028246143091801260024002D02D04E74A8
:100B3000103102E0FF3151314C700F700A61CB70FF
:100B4000022B00D10C710522D20185182A7C012AC2
:100B500006D02E74006801F001FE20462C74F8BD0A
:100B60000220F8BD10B54C07640F28216143091815
:100B7000FF3151318B614A610022CA614A700C70A9
:100B8000006802F013F8002010BD70B54B07027921
:100B90005B0F934201D9012070BDCD0900240122D1
:100BA000002D05D02821594309184A74103105E059
:100BB000282569430918FF3151314C708A700B7038
:100BC0000523DB01C5182B7C012B06D02A74006895
:100BD00001F0D0FF2C74002070BD022070BD70B5F4
:100BE0004C07640F2821614309188B624A62012275
:100BF00034256A540B630023CB624A740C7400687A
:100C0000103101F0D3FF002070BD000070B5044624
:100C1000006802F061FA010403D5204600F006FDE9
:100C200070BD41050DD5206840308188464A11408D
:100C30008180204600F0FCF80021204600F02AF9CF
:100C400070BD410404D52068403081883F4A78E077
:100C5000810404D52068403081883D4A71E00B2131
:100C60008901C504042208236118002D1ADA2068BE
:100C700040300588954305802068403002889A43BB
:100C80000280087A012805D100200872014620461A
:100C9000FFF798FC204600F0DFF82068403081889C
:100CA0002C4A4EE0050510D52068403001881943D4
:100CB0000180206840308188274B1940818020685E
:100CC00040300188114301800AE0050627D52068DD
:100CD000403085888026B5438580087A002803D077
:100CE000204600F00BF970BD2068403005881543A0
:100CF00005802068403002881A4302800120087273
:100D000020684030808A3C21800808400521C901C4
:100D10006118C86401212046FFF754FC70BD8105AD
:100D200009D52068403081880C4A114081802046D6
:100D300000F0A8F870BDC005FCD52068403081885F
:100D4000074A1140818070BDFFFB0000FFBF00001B
:100D5000FFDF0000FFEF0000FFF70000FFFD0000D5
:100D6000FFFE0000F8B5040007D00520C0012618DA
:100D7000707C0025002802D005E00120F8BD357404
:100D8000204600F039F803207074206801F0AAFEB4
:100D9000002001270AE02821414309194F740874F3
:100DA000CD740D624D62401CC0B28D6221798142CA
:100DB000F1D800220FE02820504300190146FF31EE
:100DC00041314D740A74FF300130CD7405664566BB
:100DD000521CD2B2856620799042ECD807CC0C3CEC
:100DE00001F076FE25737774A07A012802D120469F
:100DF000FFF7D2FB0020F8BD08B500680A49884219
:100E000010D10A48C2690121C9050A43C261C069FB
:100E100000220840009011461F20FFF7B9FB1F2059
:100E2000FFF7AAFB08BD0000005C00400010024074
:100E300070B5044640790125022801D0FFF756FA23
:100E40000520C00124182946A06D01F027FAA06DE5
:100E500001F0E5F970BD000010B50446407A0028A5
:100E600006D00748016906229143016100F0A8FD00
:100E70000520C0012018806D01F0F8F910BD0000B8
:100E800000ED00E0052110B5C9014018806D01F0AA
:100E9000F7F910BD10B50522D2018418227C012A71
:100EA00008D0012222740173006802F02DF900209D
:100EB000207410BD022010BD052110B5C9014118D4
:100EC0008A6D5321C9004118104601F0F4F910BD94
:100ED00070B504460520C0012518287C01280AD0D9
:100EE00001202874206802F0E5F8206801F0E8FD90
:100EF0000020287470BD022070BD000010B50446AB
:100F00000520C0012018806D01F019FA607A0028D0
:100F100004D00348016906221143016110BD00009D
:100F200000ED00E0F8B505460068394CC00352D525
:100F3000E0690026C00007D4E16920040143E161B3
:100F4000E16901400126009132480168C90510D4C9
:100F50000168821511430160FFF7B4FA074604E007
:100F6000FFF7B0FAC01B642824D82A480068C005DF
:100F7000F6D5206A03273F02384020D069683940FF
:100F800081421CD0206A226AB843012109040A4325
:100F90002262226A8A4322622062C0070FD0FFF7D2
:100FA00091FA009008E0FFF78DFA0099411A1A486B
:100FB000814201D90320F8BD206A8007F3D5206A59
:100FC0006968B84308432062002E04D0E16901201B
:100FD00000078143E1612878C00705D0206BA9682C
:100FE00080088000084320632878800605D5206BA0
:100FF00010218843E968084320632868800305D5E9
:10100000206B802188432969084320630020F8BDB4
:10101000001002400070004088130000F8B50F4631
:10102000060059D03A4D2868C007C00FB84209D20F
:10103000286840084000384328602868C007C00F6F
:10104000B84249D13068334C81070CD5400704D5EC
:10105000606807210902084360606068F0218843E6
:10106000B168084360603078C00726D070680128F6
:101070000ED0216802280ED0890700292CDA616879
:101080008908890001436160FFF71CFA00900DE0B8
:1010900021688903F1E78901EFE7FFF713FA009967
:1010A000411A1D48814201D90320F8BD60680C2116
:1010B0000840716889008842EFD12868C007C00FD6
:1010C000B8420BD928684008400038432860286897
:1010D000C007C00FB84201D00120F8BD30784007EA
:1010E00006D56068072109028843F16808436060FB
:1010F00000F018F86168094A0906090F515CC840F8
:10110000074908600320FFF7FBF90020F8BD000045
:1011100000200240001002408813000088320008BE
:10112000B000002010B50F494B680C201A46024051
:101130000D48042A14D0082A12D19A020B4C120F1F
:10114000A45CC96A094A0907090F1032525CD90325
:10115000890F00231946FFF701F8214601F0F8FF37
:1011600010BD00000010024000127A006832000832
:10117000FEB5040071D02078DC4DC00749D0686806
:101180000007800F012820D068680007800F022820
:1011900004D16868C003800F022816D0012062685D
:1011A0000004012A18D08100002A01D0052A17D096
:1011B0002A6882432A60286888432860606800287B
:1011C0001BD0FFF77FF9064613E02868800320D57F
:1011D00060680028CED01CE0296801432960EDE753
:1011E0002A680A432A60F7E7FFF76CF9801B642836
:1011F00070D828688003F7D50BE0FFF763F906463F
:1012000004E0FFF75FF9801B6428F1D828688003A9
:10121000F7D420780126800700283EDA68680007A6
:10122000800F13D068680007800F022804D1686817
:10123000C003800F012809D0E068002828681DD06D
:1012400030432860FFF73EF907460CE02868800726
:101250000CD5E068012800D108E043E1FFF732F93E
:10126000C01B0228C4D828688007F7D52868F82151
:1012700088432169C900084328600EE04008400007
:101280002860FFF71FF9074604E0FFF71BF9C01BB2
:101290000228ADD828688007F7D42078000722D527
:1012A000E0690028686A0ED030436862FFF70AF9E7
:1012B000074604E0FFF706F9C01B022898D8686AC1
:1012C0008007F7D50FE0400840006862FFF7FAF8A2
:1012D000074605E09DE0FFF7F5F8C01B022887D818
:1012E000686A8007F7D4207804274007002860DA6E
:1012F00000200190E869C00008D4E969B8060143FC
:10130000E961E96901400120009101907848016894
:10131000C90511D40168821511430160FFF7D2F8A5
:10132000009005E0FFF7CEF80099401A642870D8C5
:101330006F480068C005F5D5A06801280AD00028CC
:1013400001D0052810D0286A400840002862286A89
:10135000B84301E0286A30432862A068002812D010
:10136000FFF7B0F800900AE0286A38432862F1E7F6
:10137000FFF7A8F80099411A5E48814249D8286AC7
:101380008007F5D50DE0FFF79DF8009006E0FFF728
:1013900099F80099411A574881423AD8286A80073B
:1013A000F5D40198002804D0E86901210907884391
:1013B000E8612078C00635D5606901280CD0401D51
:1013C000686B23D038436863686B400840006863EB
:1013D000FFF778F8064622E0686B38436863686B6D
:1013E00030436863FFF76EF8064604E0FFF76AF8DB
:1013F000801B02285BD8686B8007F7D5686BF821E3
:101400008843A169C900084368630BE0B843686377
:10141000F4E74CE0FFF756F8801B022847D8686BCA
:101420008007F7D4206A00285ED069680907890F11
:10143000022942D0012636060228286805D0B0438A
:101440002860FFF73FF8044633E0B0432860FFF719
:1014500039F8074604E0FFF735F8C01B022826D804
:1014600028688001F7D4E86AE16A000900010843AE
:10147000E862616AA06A084369687B22D2039143EB
:1014800008436860286830432860FFF71BF804466B
:1014900004E0FFF717F8001B022808D8286880012D
:1014A000F7D521E0FFF70EF8001B022801D9032031
:1014B000FEBD28688001F5D416E00128F8D06868E0
:1014C000E96A0322D203636A02409A420AD10907F9
:1014D000E26A090F914205D10F2189040840A16AEF
:1014E000884201D00120FEBD0020FEBD0010024058
:1014F0000070004088130000094910B5401E884262
:1015000001D9012010BD074C60610321081F01F0C3
:1015100045FE0020A06107202061002010BD0000D2
:10152000FFFFFF0000E000E0FEE770B500231D466E
:101530000EE0040F0A2C02D25E00303401E05E009F
:1015400037348C555C00641800015B1C6570DBB29D
:101550009342EED370BD000070B586B0142168468A
:10156000FEF744FE19484269012189050A43426198
:1015700042690A400592426949110A43426142693F
:101580000A400592426949000A43426140690024C9
:1015900008400590FD200926F60600900194694652
:1015A00002943046FEF7B6FE0120022501906946FE
:1015B000009502943046FEF7ADFE0194694604485A
:1015C00000950294FEF7A6FE06B070BD0010024022
:1015D0000004004810B500220F49104800F0CCFC70
:1015E000002801D0FEF782FE0D490C4800F0CEFE27
:1015F000002801D0FEF77AFE0A49084800F0ABFA4D
:10160000002801D0FEF772FE044800F039FF0028E0
:1016100001D0FEF76BFE10BD0000002090010020FD
:10162000B800002090000020FEE70000FEB5044650
:10163000ACE18A8817073F0F31D0BE00815B019172
:1016400009047CD5815BD64A114080221143815325
:10165000282078430519FF355135287B00286FD0A5
:10166000E87802286DD0287822688100505ACD4B46
:101670001840CD4B18435052297820688A00825A6E
:1016800052047DD55022125ACB00C849121859185D
:10169000515A8905890D009173D02A89DBE0D20661
:1016A0002CD40188BF4A803A11400122D203114351
:1016B000018020682546103501464030028A207C92
:1016C0005218C100B9480818105A8005800DE06210
:1016D000616A0818606200212046FEF791FF207BB6
:1016E0000028A5D0A8690028A2D1207B802108432A
:1016F0002168403188810020207347E12546FF356D
:1017000002885135130520D5098A09182878C200A6
:10171000A648001D1018085A532183059B0DEB6144
:10172000C900EA886118206801F0D9FC216808889E
:101730009B4A1040802210430880204602E0A6E029
:1017400065E074E0FFF7B8FB20E11104D5D501880E
:10175000934A1140802211430180206801464030A5
:10176000028A2878914E5118C000361D8019085AF7
:1017700083059B0DEB6111D0696900290ED001E052
:101780005CE05AE0EA88206801F0A9FCE969686930
:101790004018686100212046FEF73EFF206801885E
:1017A0000A05AAD48904890F0329A6D05021095A11
:1017B0000818801901888905890D01802969002987
:1017C00008D03E290AD84A08C90700D0521C01880F
:1017D00092020CE001880122D20308E04A09C906FE
:1017E00000D1521E018892020123DB031A431143E8
:1017F0000180216808886E4A10400122120350407F
:1018000052005040684A403A10430880BEE02068C9
:101810005021095A0A182978CB006449091D591822
:10182000515A8905890D009119D0EA8813E029469B
:101830002046019AFEF74AFF009010E05022CB00AC
:10184000125A5A491218091D5918515A8905890DF9
:10185000009104D06A896969009B01F040FCE86945
:1018600000994018E8616969009808186861A869DA
:10187000002803D029690098814204D9297820469C
:10188000FEF7CAFE03E02946206801F08FF90198AF
:1018900000067BD5282023684743985B3919414AC5
:1018A000803A10400122D20310439853C87C103173
:1018B00001281DD00198C00564D420685022125A16
:1018C00013180878394AC0008018185A8A698005A8
:1018D000800D82424FD9121A8A614ED04A6912187D
:1018E0004A61CA691018C861206801F05FF94DE0CB
:1018F000002088610B7B002B3FD0019B5B0617D536
:101900004B78002B02D0012B09D036E02068502301
:101910001B5A18180B78DB001B18244817E02268A4
:1019200050239B5A9A180B78DB009B181F4A1FE024
:101930004D782368002D02D0012D11D01DE05020DC
:10194000C05AC0180B78DB001B181848001D181867
:1019500003889B059B0D03800388134303800CE0E1
:101960005022D25AD2180B78DB009B180F4A121D56
:101970009A18108001E00020886109782046FEF75F
:101980003FFE03E02046019AFEF710FF2068014663
:1019900040318A88120400D54BE60020FEBD0000CD
:1019A0008F0F00008F8F0000C08000000204000035
:1019B0008FBF00007047704710B5FEF789FD10BD5E
:1019C00030B595B030216846FEF710FC00240C9429
:1019D0000D940E94142110A80F94FEF707FC01201B
:1019E0000190009000040990000102250A900895DA
:1019F0000B946846FFF7BCFB002801D072B6FEE7E7
:101A000007200C900E9401210D950F940CA8FFF760
:101A100005FB002801D072B6FEE7012040041090BB
:101A20008020149010A8FFF77DFA002801D072B62C
:101A3000FEE715B030BD70470522D2018018806BDB
:101A40000021403001740846704770B505460520F6
:101A5000C0012A18946BD26B6178D26820789047C5
:101A6000402322460121284600F0CFFB002070BD14
:101A700070B50446812100F0BBFA00250121204603
:101A8000E56200F0B5FAFF206D3005510520C00178
:101A90002418A06B002806D0E06B80688047A06BFC
:101AA00000F057FEA563002070BD052110B5C901E7
:101AB0004218946BE06C012806D1D26B6178D26831
:101AC000207890470020E064002010BD0A210180AA
:101AD000004870478001002029210180004870479C
:101AE000F000002029210180004870471C010020DF
:101AF00029210180004870474801002070B5044644
:101B0000002640230322812100F072FB012540239F
:101B1000032229462046E56200F06AFBFF206D3073
:101B20000551542000F016FE0521C9016118886393
:101B300000280ED00546002240300274C86B406871
:101B4000804740232A460121204600F05EFB3046B4
:101B500070BD0126FBE702460220002904D00520C3
:101B6000C0011018C16300207047134610B505224C
:101B7000D2018418A26B247F032C0BD14032147C39
:101B8000002C01D0012010BD012414740A468121CB
:101B900000F0DEFB002010BDF8B505460520C001B1
:101BA0002B1800226E46986B32800E786027944680
:101BB00014463E4023D0202E55D14A78921E130061
:101BC00001F0DEFA0A11095151515151150D06511A
:101BD000897801644BE001220146403135E04988B3
:101BE000090A416443E00122014644312DE001220B
:101BF000C264CA880146284600F063F837E04E7890
:101C0000002E06D0062E0AD00A2E22D00B2E2AD164
:101C100026E0187F032826D10222694615E048886D
:101C2000000A222802D0212808D00DE0CA883F2AC5
:101C300000D93F22D86B0068844605E00E48CA8868
:101C40008446092A00D909226146284600F056F840
:101C50000DE01A7F032A06D1012201464831F4E73C
:101C60001A7F032A05D0284600F021F802242046D6
:101C7000F8BD89788164FAE774010020052210B567
:101C8000D2018218526B52689047002010BD134653
:101C900010B50A46002100F0B8FA002010BD134626
:101CA00010B50A46002100F053FB002010BD10B50E
:101CB0000446802100F02FFB0021204600F02BFB82
:101CC00010BD10B50524E401032304196361C31D8D
:101CD000F933DA651A6613460A46002100F095FAD0
:101CE000002010BD052110B5CA01821800235161E2
:101CF0001A46194600F089FA002010BD10B50524D7
:101D0000E401022304196361C261134602620A46B8
:101D1000002100F01DFB002010BD052210B5D201EE
:101D200004218218002351611A46194600F010FB65
:101D3000002010BD10B50A46024903A000F0ECF8DF
:101D4000004810BD54040020437573746F6D204823
:101D5000494420436F6E66696700000012200880C6
:101D6000004870472000002010B50A46024903A031
:101D700000F0D2F8004810BD54040020437573747D
:101D80006F6D2048494420496E74657266616365D1
:101D90000000000004200880004870471C0000205C
:101DA00010B50A46024903A000F0B6F8004810BD7D
:101DB0005404002053544D6963726F656C656374FD
:101DC000726F6E696373000010B50A46024903A082
:101DD00000F0A2F8004810BD5404002053544D33C5
:101DE0003220437573746F6D2048756D616E206984
:101DF0006E746572666163650000000010B51A209C
:101E000008800948046BC16A406B081809D0082291
:101E10000649FFF78AFB0549042210312046FFF7E7
:101E200084FB0248801E10BD80F7FF1F3600002093
:101E3000F8B50D46044600206946088069880520EB
:101E40000A0AC0012018130001F09AF90844050B92
:101E5000184444384144006B237C026869461846A4
:101E600017E0217C0226406B002905D0C16A684634
:101E700088470146467039E0816AF8E7C9B20B002D
:101E800001F07EF90604091013161928006B426848
:101E900003E0904719E0006B8268002A1AD0207C8A
:101EA0006946F6E7006BC268F7E7006B0269F4E782
:101EB000006B4269F1E7006B8269EEE7217C002943
:101EC00008D1406B416B6846884701460EE0217C93
:101ED000002904D029462046FFF7E9FEF8BD406BF3
:101EE000016B6846884707220146427068460088B1
:101EF00000280AD0EA88002A0AD0824200D9024685
:101F0000684602802046FFF7F9FEE8880028E5D100
:101F10002046FFF702FFF8BD70B5002300281DD052
:101F20000446002502E06D1CEDB2641C2678002EEC
:101F3000F9D16C00A41C14801278CA5403225B1CD3
:101F4000CA5400245B1C06E0CA545B1CDAB28C54F1
:101F5000521CD3B2401C0278002AF5D170BD014654
:101F60000020002904D0012901D0022901D002203B
:101F7000704701207047000010B5002811D00523DC
:101F8000DB01C3185C6B002C01D000245C630029CA
:101F900000D0196301211977027000F0DFF80020EA
:101FA00010BD05A001F0CAF805A001F0C7F80AA00D
:101FB00001F0C4F8022010BD4552524F523A2000A1
:101FC000496E76616C696420446576696365206852
:101FD000616E646C650000000A000000052210B507
:101FE000D2018018006CFEF747FBFFF7B8FF10BD69
:101FF000052210B5D2018018006CFEF71BFBFFF71D
:10200000AEFF10BDF8B506460520C00134181346D2
:10201000002908D0606B4269002A02D0207F032883
:102020004FD00220F8BD354660691435022804D02F
:10203000042839D0002837D03AE02F69E868B84240
:1020400007D9C01B82B2E86019463046FFF727FE69
:1020500012E0AD6839462846FEF76AF8002912D129
:10206000BD4210D3A06985420DD2002211463046F0
:10207000FFF715FE0020A06100231A4619463046DE
:1020800000F0C3F814E0606BC168002904D0207F21
:10209000032801D1304688478021304600F03BF9C3
:1020A0003046FFF71FFE03E08021304600F033F991
:1020B0001520400130180178012904D10021017058
:1020C00001E0304690470020F8BD70B50546052078
:1020D000C0012B181646002908D0586B8269002AC7
:1020E00002D0187F03282DD0022070BD2C46FF346B
:1020F00058695534032802D005281CD024E0E16833
:10210000206981420AD90B1AE360834200D3034657
:102110009AB231462846FFF7BAFD15E0586B0169BF
:10212000002904D0187F032801D128468847284673
:10213000FFF7F3FD08E0002001465861284600F053
:10214000EAF801E028469047002070BD052210B54E
:10215000D2018018006CFEF7D5FC10BD10B51949EE
:1021600005228865D201841817491848216408603F
:102170000820087102204871C871002048728872D6
:10218000C8720846FEF7EEFD002801D0FEF7AEF853
:10219000002218231146206CFEF715FA582300225E
:1021A0008021206CFEF70FFA982300228121206CF9
:1021B000FEF709FAD82300220121206CFEF703FA6A
:1021C000002010BD6C090020EC060020005C0040DF
:1021D000CA094906490E282359431B01C018006C3F
:1021E0000818002A01D0807C7047FF304130FAE7A0
:1021F00010B51C460523DB01C0181346006C2246AF
:10220000FEF789FCFFF7ABFE10BD10B50524E40115
:102210000019006CFEF7A6FCFFF7A1FE10BD70B51B
:102220000022044640231146FFF7E2FFE01D40264E
:10223000F930012546668565334600228021204617
:10224000FFF7D6FF0520C00166622018A56105775B
:102250000021416161604162816B002904D0406BC3
:102260000021426820469047002070BD0521C90129
:102270004018017F042901D1417F01770020704778
:10228000052110B5C90141180A7F032A04D1496B01
:10229000C969002900D08847002010BD01740020C2
:1022A0007047052210B5D2018018006CFEF7F2FDD0
:1022B000FFF755FE10BD70B505465520C000281823
:1022C000044600F04FF80520C001012128184161A3
:1022D000C18D8161152040012818007AC106C90E00
:1022E0000AD001290DD0022910D0C109C901284600
:1022F00000F011F8002070BD2146284600F0C5F816
:10230000F8E72146284600F0FAF9F3E72146284687
:1023100000F040F9EEE7052210B5D2018018006CFC
:10232000FEF733FCFFF71BFE10BD052110B5C901F8
:102330004018006CFEF7CCFDFFF711FE10BD052123
:10234000C9014018017F41770421017700207047BF
:1023500010B50524E4010019006CFEF740FCFFF7FE
:10236000FEFD10BD0A7802704A784270CB788A78F8
:102370001B02D21842804B790A791B02D218828044
:102380008A79C97909025118C1807047024610B58F
:102390000020002904D00523DB01D218516310BDB1
:1023A00005A000F0CBFE06A000F0C8FE0AA000F0D9
:1023B000C5FE022010BD00004552524F523A200087
:1023C000496E76616C696420436C61737320686147
:1023D0006E646C65000000000A000000052210B564
:1023E000D2018218526B0224002A04D0126890474E
:1023F000002800D10024204610BD000070B50E4614
:1024000089781E4C05462170012904D93146284699
:10241000FFF74DFC70BD0520C0012818027F022A7D
:102420000AD0032A0ED031462846FFF740FC217817
:102430002846FFF723FC70BD002913D003226960F2
:1024400002770AE0002911D0686888420AD0C1B238
:102450002846FFF713FC217869602846FFF7BEFF86
:102460000228D3D02846FFF758FC70BD022202771D
:1024700028466960FFF702FCF4E70000B400002082
:1024800010B5FFF752FF002010BDF8B500220092F2
:102490000A7860231A400523DB01C518002A07D0FB
:1024A000202A01D0402A6AD16A6B9268904768E07E
:1024B0004C7800220126230000F062FE0A3F5A6198
:1024C00055610906612C2961FFF7B2FC59E0044609
:1024D0008888002819D1C888002816D14888802803
:1024E00013D24706287F7F0E03280ED0AF773946D8
:1024F0002046FFF7D6FE2046FFF70FFC002F02D044
:10250000022028773DE02E773BE0204637E0FFF7BA
:1025100075FF36E0CB88012B31D12B7F012B04D006
:10252000022B02D0032B2AD104E082600122014653
:10253000083115E00122011D12E02A7F012A03D093
:10254000022A01D0032A1AD1CA88022A17D1C660EA
:10255000696A002901D00321C160014602220C31C1
:10256000FFF7CCFB0DE0498801290AD16E620EE02D
:102570002B7F012B07D0022B05D0032B03D0FFF7B5
:1025800096FB0098F8BD49880129FAD16A62FFF7E5
:10259000C4FBF6E7F8B50A461378044660201D46EA
:1025A00005400520C001002709792018002D09D019
:1025B000202D01D0402D77D1406B114683682046F5
:1025C00098479AE05B069B0F012B07D05378002BAE
:1025D0003BD0012B2BD0032B66D105E0406B11467D
:1025E000836820469847F8BD007F022802D0032860
:1025F0007FD10BE000297CD080297AD02046FFF7DC
:102600008AFE80212046FFF786FE76E0508800286B
:1026100009D1002907D0802905D0D088002802D10F
:102620002046FFF778FE2046FFF777FB65E0007F46
:102630000228DFD003285CD1508800285DD14806ED
:10264000F1D02046FFF7CAFCEDE7007F0026022804
:1026500002D003284DD116E0002901D0802948D1AD
:10266000C80906D04806400E142148430119143108
:1026700006E04806400E142148430119FF31553148
:1026800002220E6031E0C8090FD00807000F1423A2
:1026900058430019806900282BD04806400E1422A8
:1026A00050430519143511E023E00807000F1423E7
:1026B00058430019FF300130806D002819D04806BA
:1026C000400E142250430519FF355535002909D015
:1026D000802907D02046FFF77BFD002802D001208B
:1026E000286000E02E60022229462046FFF706FB04
:1026F00003E011462046FFF7DAFA3846F8BD70B518
:1027000005460C4608786021084003D0202801D0F7
:10271000402818D10520C0012818017F012903D0C5
:10272000022901D003290ED1217901290BD8406B50
:102730002146826828469047E188014307D1284610
:10274000FFF7EBFA03E021462846FFF7B0FA002036
:1027500070BD70470048704794060020F0B5002215
:1027600094460A789400035B924A1340CA78002A80
:102770005ED0012A63D0022A03D0032A5BD0012253
:1027800094468D4A134303530D78AE00845B8B4B04
:102790001C402C4314438453884D0E7B0446303533
:1027A0004034002E4ED0CE78022E0E7872D0B70074
:1027B000C65BBE46824F3E4016437746C653268AC6
:1027C0000F783618FF00BF190126B602BE190F890F
:1027D0007F087F003780248A0E782418F600361987
:1027E000784C34194E897608760026804C78002C77
:1027F0000C7875D0A600845B640404D5845B724FAA
:102800001C403C4384530C78A600845B640605D5C9
:10281000845B1C40684B40331C438453CB78012BB2
:102820000B787DD09C00035B2B4020256B40B5E0EE
:102830000122520201E0032252021343A1E70122C6
:102840009202FAE74E78002E25D0248A0E782418BA
:10285000F60036190124A4023419CE8876087600D1
:1028600026800C78A600845B640605D5845B1C403A
:10287000514B40331C438453CB78012B05D009784E
:102880008B00C15A294020244EE009788B00C15AA0
:1028900029408BE056E0258A0E782D18F60076192F
:1028A000484D7519CE88760876002E80248A0D78DA
:1028B0002418ED002C19434DAD1C64192588AD0575
:1028C000AD0D258001270E69FF03002E09D03E2E95
:1028D0000BD87508F60700D06D1C2688AD020BE0FA
:1028E00037E025883D43258008E07509F60600D1CC
:1028F0006D1E2688AD023D432E4326800C78A50030
:10290000445B640404D5445B1C402F4B1C4344537C
:10291000097800290AD08B00C15A2B4CF13C00E009
:1029200039E021400124640361403FE00188264BE7
:10293000F13B194001231B0359405B0059401143EF
:10294000018035E0B700C65BBE46204F1E403E43C7
:1029500033E7A600845B640404D5845B1A4F1C40F3
:102960003C4384530C78A600845B640605D5845BE5
:102970001C40114B40331C4384530B789C00035B79
:10298000114EF13E3340012636037340760073400A
:102990001343035379E79C00035B2B40134303531A
:1029A00009788B00C15A084CF13C21401143C152B7
:1029B0006046F0BD8F890000808000008F8F00008E
:1029C0008F8E00000404000080C0000080810000A1
:1029D000F0B50A780F7B374B4E78374D374C920065
:1029E000002F22D0002E865A41D0760403D5865A75
:1029F00026402E4386520A789600825B520605D501
:102A0000825B2C4F224040373A4382530A7896002B
:102A1000825B22402A4382530A789400025B274D4E
:102A200030352A401A43025317E0002E0ED0855A43
:102A30006D0605D5855A25401E4C403425438552E8
:102A400009788A00815A1D4C30340BE0865A76048E
:102A500003D5865A26402E43865209788A00815A29
:102A6000154CF13C2140194381520020F0BD760401
:102A700003D5865A26402E4386520A789500425B3B
:102A8000520605D5425B0B4E22404036324342533C
:102A90000A789500425B2240064C40342243425360
:102AA0000A789400025B044DF13D2A401A43025318
:102AB000C6E700008080000080C000008F8F00000B
:102AC0004030018B0122D203114301830020704763
:102AD000012140300180002101808180018208466F
:102AE000704700004030034902888A43028000207A
:102AF0007047000080BF000030B50A7B002A30D14B
:102B00004A78194D002A194B0A7814D09400025BB8
:102B1000520605D5025B2A40144D40352A43025324
:102B2000CA78012A1DD009788A00815A0E4C3034A7
:102B30002140202412E09400025B520404D5025B81
:102B40002A400B4D2A43025309788A00815A084CC7
:102B5000F13C214001242403614064006140194399
:102B60008152002030BD00008F8F00008080000067
:102B700080C0000010B54A780978094B8900002A06
:102B8000425A03D0074C2240102403E0064C224056
:102B90000124240362401A434252002010BD000069
:102BA00080800000BF8F00008FBF0000F0B50D4691
:102BB0004B780746FE4A097B40370446012B08D074
:102BC00000296FD0E87802286DD001286CD0012050
:102BD000F0BDAE692869864200D90646002912D0A8
:102BE000E97802291FD0286A801B28622878810092
:102BF000615A4906398A6ED50919C0004118ED4855
:102C00000818068018E1B3B2EA882046696900F026
:102C100082FA388A29780019C9000918E548001F86
:102C2000081806800EE1296A8142287874D981004B
:102C3000605A1040E04A10436052286A801B2862A4
:102C400028788100615A4906697878D5002902D030
:102C500001292AD030E0398AC00009194118D54825
:102C6000081801888905890D0180002E08D03E2EA4
:102C70000CD87108F20700D0491C028889020EE0C6
:102C800001880122D2031143018015E07109F20687
:102C900000D1491E028889020123DB0319430A433C
:102CA000028009E0F9E024E1A4E13A8AC0001119A8
:102CB0004118C048081806806A89B3B2204669697D
:102CC00000F029FA6869801968612969286A8842D0
:102CD00002D9801B02E0D8E006460020286268780E
:102CE000002802D001282BD030E0388A297800193A
:102CF000C9000918AF48001F081801888905890D07
:102D00000180002E09D03E2E0DD87108F20700D0A8
:102D1000491C028889020FE0A4E001880122D20345
:102D20001143018012E07109F20600D1491E0288A8
:102D300089020123DB0319430A43028006E007E00E
:102D4000388A29780019C9000918A1E02A8974E095
:102D5000002902D0012928D02FE0398AC0000919A2
:102D600041189448001F081801888905890D0180C1
:102D7000002E08D03E2E0CD87108F20700D0491C56
:102D8000028889020EE001880122D20311430180EA
:102D900013E07109F20600D1491E0288890201235D
:102DA000DB0319430A43028007E0398AC00009198E
:102DB00041188048001F081806802A89B3B22046AF
:102DC000696900F0A8F96869801968612969286A49
:102DD000884201D9801B01E00646002028626878FD
:102DE000002802D0012837D026E0388A2978001937
:102DF000C90009186F48081801888905890D0180E4
:102E0000002E08D03E2E0CD87108F20700D0491CC5
:102E1000028889020EE001880122D2031143018059
:102E20000AE07109F20600D1491E028889020123D5
:102E3000DB0319430A4302806A89B3B220466969F9
:102E400000F069F928788100605A594A3032104000
:102E500010225040202215E1398A08192978C9002A
:102E60000918CCE68200A05A544B1840544B184322
:102E7000A052388A2A780019D20012184D488BB215
:102E8000001F101803802A89D8E70919C0004118CB
:102E90004848001F0818068058E7A9692869814238
:102EA00001D9091A01E008460021A961398A2A7866
:102EB0000919D20052183F4951180A889205920DFB
:102EC0000A8000287ED03E2807D84208C00700D0DC
:102ED000521C088892021043CAE04209C00600D181
:102EE000521E0B8890020122D203104303430B8031
:102EF000BFE0002B28D1388A29780019C9000918A9
:102F00002C48001F081801888905890D018029694E
:102F100000290AD03E290CD84B08C90700D05B1CF9
:102F200001889B02194301800EE001880123DB0325
:102F3000F8E74B09C90600D15B1E068899020123F8
:102F4000DB0319430E4306806878002802D001286D
:102F500047D027E0388A29780019C9000918154890
:102F6000081801888905890D0180296900290AD07E
:102F70003E290CD84B08C90700D05B1C01889B0276
:102F8000194301800EE001880123DB03F8E74B09B8
:102F9000C90600D15B1E068899020123DB03194391
:102FA0000E430680E869002863D0287881000AE093
:102FB0008F8F000006040000808100008F8E0000CB
:102FC0008080000050E0605A430401D5430602D4DB
:102FD000344B18424DD1605A1040334A104360526E
:102FE00047E0398A08192978C90009182F480818B4
:102FF000298AC6E7A9692869814201D9091A01E02D
:1030000008460021A961002B27D1398A2A7809199D
:10301000D20052182549091F51180A889205920DAD
:103020000A80002808D03E280CD84208C30700D0E8
:10303000521C0B8892020EE00A880123DB031A431C
:103040000A800AE04209C30600D1521E0B88920290
:103050000126F603324313430B806978002900D11F
:1030600024E7012915D004E008880122D20332E7C1
:10307000088028788100605A0D4A1040012212030E
:10308000504052005040084A403A104360520020DD
:10309000F0BD3A8A11192A78D20052180349511802
:1030A000E6E7000040400000C08000000604000089
:1030B0008FBF000000214030818002490180002044
:1030C0007047000080BF000010B50248FDF79EFD6C
:1030D00010BD0000EC06002040308088704780184A
:1030E00010B5012292025C088018002C07D00288DB
:1030F0000A70120A4A70801C891C641EF7D1DA0714
:1031000001D00088087010BD002902D18021403014
:10311000818100207047801801225B1C920210B54B
:103120005B088018002B08D04A780C7812022243E2
:103130000280801C891C5B1EF6D110BD10B5024AAE
:10314000024900F05CF810BD1D3200088C0100201F
:10315000F8B5040C8BB2264682B25E430D0C1046C5
:10316000370C5843360480190021794116466E43C6
:10317000370C36048019794126466E438919F8BD0B
:1031800030B47446641E2578641CAB4200D21D46E0
:10319000635D5B00E31830BC184700008307FF2223
:1031A000DB0E9A408907090E9940002808DB830846
:1031B00009489B001B181868904308431860704723
:1031C0000007000F0838830804489B001B18D869C3
:1031D00090430843D861704700E400E000ED00E050
:1031E00002E008C8121F08C1002AFAD170477047D0
:1031F000002001E001C1121F002AFBD17047F8B581
:1032000016460F460446002503E03946B047641CC5
:103210006D1C20780028F8D12846F8BD38B5044642
:103220006846047069460320ABBE204638BDFDF7F2
:1032300057F9FEF7C5FBFEF78FF9FEF7CBF9092525
:10324000ED06FF24F534012202212846FDF734F96A
:103250002046FDF74DF8002202212846FDF72CF903
:103260002046FDF745F8EEE70203040506070809C6
:103270000A0B0C0D0E0F10100102030405060708BF
:10328000090A0B0C0D0E0F100000000000000000DA
:103290000102030406070809B832000800000020F4
:1032A00090010000480200089433000890010020BB
:1032B000380C0000F0310008135D1D1B0895041A3E
:1032C000A1041AC9041AFD041A35041A6904170462
:1032D00003090412013202164083045057260201EA
:1032E000020301031A1A03100E05010906A10105C4
:1032F0000719E029E715281A2501750195088102AB
:1033000095017508810395057501050819012905C1
:103310009112180803910395067508261A65301155
:103320001429658112C022501420A3021B089F0497
:103330001AA90441197311820453127A13FD1A1B3E
:103340000871044B991B241AAB0C1A39041A4B044C
:10335000C11AE5101AD9041AF1041ACD041409028D
:10336000291301011CC03209522A02C91509211171
:10337000011401223F1607058103402D05070501B1
:1033800007291A09562C691A31130A0632022A40F3
:04339000E441000014
:04000005080000C12E
:00000001FF
